:100000005FC0DAC176C075C074C073C072C071C001
:1000100070C06FC06EC06DC06CC06BC06AC069C07C
:1000200068C067C066C0040309041E036E00650053
:10003000770069006F00690074002E0063006F0094
:100040006D002E00610075001A0346005300690020
:100050006D004500780074002E0031003100300042
:1000600030001201100100000008C016DC0500037A
:100070000102000109022200010100804B09040075
:10008000000103000000092101010001222A0007EC
:1000900005810308006405010905A1010901A1000A
:1000A0000930093115002502750295028102C0054B
:1000B000091901290415002501750195048102C063
:1000C00011241FBECFEDCDBF10E0A0E6B0E0EEE3FF
:1000D000F7E002C005900D92A236B107D9F710E003
:1000E000A2E6B0E001C01D92AB39B107E1F7AED294
:1000F00024C386CF1F93162F20916F0024FF07C0C3
:100100002091700038E823272093700003C02AE56F
:1001100020936F00212FDC01E1E7F0E08D918193C6
:1001200021501216DCF381E790E0612F41D11C5F72
:1001300010936F001F9108951F93CF93DF938091C9
:100140008000835087FDA8C090917D0020917C00A5
:100150002D3209F09FC0883009F09CC0CCE0D0E07F
:10016000C91BD109CC57DF4F83EC809364008AE52B
:1001700080936000109262008881807619F0CE0131
:1001800055D27FC09A8110926D008981882331F405
:1001900010926E002DE630E082E06FC0853019F4D9
:1001A0009093810067C0863009F04EC08B8181300A
:1001B00041F482E690E090937F0080937E0082E19C
:1001C0003FC0823041F484E790E090937F008093B9
:1001D0007E0082E235C08330F1F4992341F486E257
:1001E00090E090937F0080937E0084E029C091305E
:1001F00041F48AE290E090937F0080937E008EE14C
:100200001FC09230E1F488E490E090937F008093E7
:100210007E008AE115C0813241F486E890E0909337
:100220007F0080937E0089E00BC0823241F486E932
:1002300090E090937F0080937E008AE201C080E08E
:1002400090E4909362001DC0883069F0893019F401
:10025000909383000FC08A3049F08B3059F48BE4BF
:100260008093700007C023E830E002C02DE630E044
:1002700081E003C02DE630E080E030937F002093E2
:100280007E009F81992321F49E81981708F4892F7D
:1002900080936100109280008091600084FF4CC0C8
:1002A000809161008F3F09F447C0182F893008F012
:1002B00018E0811B809361008091640098E8892791
:1002C00080936400112361F180917E0090917F0002
:1002D00030916200212F215036FF0EC030E0A9017D
:1002E0004A595F4FFC01A5E6B0E064916D933196E9
:1002F000A417B507D1F70CC0DC0130E0A9014A59B9
:100300005F4FE5E6F0E06D916193E417F507D9F7EB
:100310002F5F3F4F280F391F30937F0020937E00BF
:1003200085E690E0612F44D01C5F1C3019F08FEF00
:10033000809361001093600084E190B39C7031F46D
:100340008150D9F71092810010927B0011E0811149
:1003500010E080916300811729F0112309F475D111
:1003600010936300DF91CF911F91089585B782604C
:1003700085BF8BB780648BBF8BE4809370008AE568
:1003800080936F000895A82FB92F80E090E041E09E
:1003900050EA609530E009C02D91822797958795A6
:1003A00010F084279527305EC8F36F5FA8F3089597
:1003B000EADF8D939D930895CF93CFB7CF93C395E5
:1003C000839BE9F7839B09C0839B07C0839B05C080
:1003D000839B03C0839B01C0A3C0DF93C0917D00BA
:1003E000DD27CC57DF4F839B02C0DF91EBCF2F93EC
:1003F0000F931F9300B32FEF03FB20F94F933F930D
:1004000010B34FEF012703FB21F93BE031C04E7FD2
:10041000012F10B3216028C0102F4D7F22600000F3
:1004200000B329C04B7F2460012F000010B32BC004
:1004300010B3477F28602AC04F7E00B320612CC0D4
:100440004F7D10B320622FC04F7B00B3206432C0B9
:10045000422700B349934FEF0000102713FB20F908
:1004600010B31C70C9F1297F91F2012703FB21F918
:1004700000B3237F89F2315058F1102713FB22F982
:1004800010B3277E79F2012703FB23F92F7C81F239
:1004900000B3102713FB24F92F7971F200C010B3B9
:1004A000012703FB25F92F7359F200C000B3102771
:1004B00013FB26F9223040F200C010B3012703FBE2
:1004C00027F9243028F64F77206810B30000F9CFC1
:1004D00010E41ABF002719C03B503195C31BD04010
:1004E00010E41ABF0881033CF9F00B34E9F02091C5
:1004F0007B001981110F1213EDCF4A81441F093679
:1005000041F10D3211F0013E29F7009382003F9135
:100510004F911F910F912F91DF91CAB7C6FD4FCF19
:10052000CF91CFBFCF91189520918200222379F3EC
:1005300010918000112369F534306AF13093800006
:1005400020937C0010917D003BE0311B30937D00B7
:1005500022C0009180000130E4F40AE54F7049F4B4
:100560003091600034FD19C000936000C4E6D0E013
:1005700018C030916F0034FD10C000936F00C0E7C9
:10058000D0E00FC02795A8F45150A9F4220F000025
:10059000F9CF4AE503C042ED01C0432FC4E1D0E0EA
:1005A00032E011B31C60939A11BB02B320E41CE04B
:1005B0005F93012756E002BB279520F4515021F4A8
:1005C000220FF9CF012756E000003B5A02BBD0F2C0
:1005D000279528F4515029F4220F0000F9CF012764
:1005E00056E0279502BB20F4515021F4220FF9CF99
:1005F000012756E02991332302BB21F6037F109196
:100600008100110FC651D04002BB11F010937B0046
:1006100010E41ABF086011B3137F402F437F5F912E
:1006200000C000C002BB11BB42BB71CFFC01808186
:100630008076803231F49181913029F081E09230DE
:1006400019F080E0089581E0089508950F931F93B5
:10065000479A8E9A969A8B9A8FE79FE4A2E18150EF
:100660009040A040E1F700C000008B982EE088E1A8
:1006700090E00FB6F894A89581BD0FBE21BD76DE3F
:100680007894B898C09AB998C19ABA98C29ABB9807
:10069000C39ABC98C49A8C98949A8D98959A969877
:1006A00005E016E0A89548DD9698859B969A80917E
:1006B0006F0084FFF7CF00939A00B09902C01093A7
:1006C0009A00B1990DC090919A00892F86958695D0
:1006D0008D5F8370880F880F937F982B90939A007B
:1006E000B29909C080919A00982F9D5F93708C7F7A
:1006F000892B80939A00B3990DC090919A00892F0D
:10070000869586958F5F8370880F880F937F982BCF
:1007100090939A00849905C080919A00806280939A
:100720009A00859905C080919A00806180939A0013
:0E0730008AE990E061E0DEDCB5CFF894FFCFFF
:02073E005AFF60
:00000001FF
